:10000000022900009030201C133086000000000000
:100010008030201C1330860000000000000000002B
:10002000000005100000D030201C133086000608A8
:10003000A6000830A619093065001330A018323028
:1000400020199030201C133086000608060400009A
:1000500000000000A600A61D05162130A100A10B7E
:100060002F2800000000093065000512A2030319C3
:100070000134000000000000000000000000012822
:100080000330A30086194028861940288619402885
:10009000861940288619402886194028A30B422833
:1000A000861D50280000060806040604A60026192E
:1000B0004028A61940280608A600261D4028000052
:1000C00000000608A600A61D40283130A100A10BA3
:1000D0006728000000000608A600261D40284E30B4
:1000E000A100A10B712800000608A600261D4028CB
:1000F0002E30A100A10B7A2820120134851DA015F5
:10010000A01DA501A50A25192010251920162519BD
:10011000A501A40AA019A40124192014A011851472
:1001200020188510051520180511000000000F305B
:10013000A100A10B992801340230A100A10B9E2837
:100140008030201C133086000230A100A10BA628AD
:10015000D030201C133086000330A100A10BAE2844
:100160009030201C1330860000000B30A100A10B42
:10017000B72801340230A100A10BBC288030201C1C
:1001800013308600000000009030201C13308600E1
:10019000000000001530A100A10BCC280530A20BF7
:1001A000BE28A2008030201C1330860006080604FA
:1001B0000000A600261DA0151330A100A10BDE280B
:1001C0009030201C1330860000000000000000006A
:1001D0000530A20BD228A2008030201C13308600EC
:1001E000000000009030201C133086001130A10068
:1001F000A10BF828A203031901340430A100A10BBC
:10020000FF28EC28093065000C30660013308600AA
:100210008514A00120142016013042290000053069
:10022000A200BA20000000000000000000007E20B4
:100230000000000000001130A200012000000000BA
:100240002011C830A2000120000000000000523040
:10025000A20001200000000020150530A2000120AE
:10026000000000000000261900009C200000000093
:1002700000000530A200BA200000000000000000CD
:10028000A20001200000201A40201030A20001200E
:100290000000000000002011A2000120A010A619FB
:1002A000A014C830A200012000000000000052305D
:1002B000A20001200000000020150530A20001204E
:0202C0000E2905
:02400E00FA3F77
:00000001FF
